:1000000090C0C4C0A9C0A8C0A7C0A6C0A5C0A4C0B5
:10001000A3C0A2C0A1C0A0C09FC09EC09DC005013A
:100020000906A1010507750195011500250109576C
:10003000810281018101094781020953810209007E
:10004000810181018101C0090222000101008003B8
:100050000904000001030000000921010100012240
:1000600029000705810308000A12011001000000A1
:1000700008C016DB270001010203013A036800658E
:1000800000680061004000680072007A002E007471
:100090000075002D006300680065006D006E00694A
:1000A0000074007A002E00640065003A00300030D1
:1000B00000300031000E034F006E0065004B0065FC
:1000C0000079005A0368006100660074006D0061E9
:1000D000006E006E00230073006F006600740077EE
:1000E000006100720065002000280077007700772B
:1000F000002E00740075002D006300680065006D1F
:10010000006E00690074007A002E00640065002F04
:10011000007E006800650068006100290004030992
:10012000040011241FBECFE5D1E0DEBFCDBF10E03B
:10013000A0E6B0E0EAE1F7E003C0C89531960D9281
:10014000A436B107D1F710E0A4E6B0E001C01D92DB
:10015000AC39B107E1F77CC153CFA82FB92F80E0AC
:1001600090E041E050EA60956F5F58F42D9138EFD0
:1001700082279795879510F0842795273F5FC8F3CE
:10018000F3CF0895EADF8D939D930895CF93CFB772
:10019000CF93C395B29BE9F7B29B18C0B29B16C030
:1001A000B29B14C0B29B12C0B29B10C0B29B0EC0D7
:1001B000C2B7C1BBC2B7D3BBD2B3C2BBCD1BC1BBDD
:1001C000D3B3C2B7C1BBCC27C2BFCEC00F92DF939F
:1001D000C0917F00DD27CA57DF4F012EB29B03C0BD
:1001E000DF910F90D9CF2F930F931F934F932FEF42
:1001F0004F6F06B302FB20F95F933F9350E03BE063
:1002000065C016B30126502952FDC89556B3012783
:1002100002FB25F92F7306B3B1F05027102712FB0C
:1002200026F906B22230F0F000C016B3012702FB17
:1002300027F90126502906B22430E8F54F772068C7
:1002400016B30000F6CF50274F7D206206B2102F64
:10025000000000C006B300265029102712FB26F923
:1002600006B2E2CF4F7B06B3206400C0DACF01268E
:100270005029167006B269F14E7F2160012F16B326
:1002800028C0002650294D7F06B22260102F29C0B9
:10029000012650294B7F06B22460012F2DC016B3D2
:1002A00001265029477F2860000006B22EC04F7EED
:1002B00006B3206130C0422706B349930026502977
:1002C000102706B24FEF12FB20F9297F16B379F2FF
:1002D000167049F10126502906B2012702FB21F9C7
:1002E000237F06B371F2002650293150D0F006B2B8
:1002F000102712FB22F9277E16B351F2012650294E
:10030000012702FB06B223F92F7C49F2000006B355
:10031000102712FB24F90026502906B22F7939F252
:1003200070CF002717C03B503195C31BD0400881C8
:10033000033CF1F00B34E1F020917D001981110FA5
:100340001213EFCF4A81441F093639F10D3211F0F3
:10035000013E39F7009384003F915F914F911F91C7
:100360000F912F91DF910F90CF91CFBFCF91189523
:1003700000918400002381F310918200112379F50C
:1003800034307AF13093820000937E0010917F0028
:100390003BE0311B30937F0024C00091820001308C
:1003A000F4F40AE54F7049F43091610034FD1AC04D
:1003B00000936100C7E6D0E019C03091600034FDC1
:1003C00011C000936000C2E7D0E010C0052710E024
:1003D00000C021C0052710E0C89508BB14C03AE54D
:1003E00001C032ED032EC0E0D0E032E017B316605A
:1003F000C29A08B317BB56E020E84FEF20FF05274D
:1004000008BB279517951C3F28F700004552B0F709
:1004100020FF0527279508BB17951C3FB8F62991A3
:100420003A9561F7097F10918300110F08BBC25004
:10043000D04011F010937D00046017B3197F402F56
:10044000497F54E05A95F1F708BB17BB48BB84CFEE
:10045000CFE5D1E0DEBFCDBF10E094B714BF479A1F
:1004600088E181BD11BD93FF0DC086B399278670C9
:100470009070892B39F080E48BBF80E385BF78943E
:100480008895F89480E285BF8BE080BD82E083BFD1
:1004900089E388BB8BB780648BBF8BE48093720049
:1004A00088E081BD78948895A8959091820019166E
:1004B0000CF0A7C080917F00E2E9F0E0E81BF109B1
:1004C000935030E050E880917E008D3209F093C067
:1004D0004AE540936100983009F08DC09081892FE2
:1004E000807609F062C080E790E03093700021814F
:1004F000222321F43093710032E04CC0253021F4E6
:1005000082818093830070C02630B1F550EC8381E6
:10051000813021F489E690E032E13CC0823021F460
:1005200087E490E032E236C08330D1F482818823C0
:1005300021F48DE191E034E02DC0813021F483EC91
:1005400090E0342F27C0823021F485EB90E03EE02C
:1005500021C0833009F048C08BE790E03AE31AC02D
:10056000813221F489E590E039E014C08232E1F56E
:100570008EE190E039E20EC0283019F485E890E071
:1005800008C0293021F48281809385002DC02A3053
:1005900031F431E0909381008093800025C02B30AE
:1005A00019F58BE4809372001FC0892F99278076FC
:1005B00090708097B1F48181813019F486E690E0E3
:1005C00004C0823049F485E690E0909381008093E6
:1005D000800081E090E007C08A3019F48381809325
:1005E000650080E090E0382F8781882321F48681A0
:1005F000831708F4382F50936400309362001092F0
:1006000082008091610084FF44C0809162008F3F2E
:1006100009F43FC0682F893008F068E0861B80939A
:1006200062000BE48091640080FD03EC8F5F809397
:100630006400A8E6B0E0E0918000F0918100962F80
:10064000915086FF08C09F3F61F0C895802D8D9323
:1006500031969150F8CF9F3F21F081918D93915029
:10066000FACFF0938100E09380007727C62F69309E
:1006700040F488E690E086DD9C2F9C5FC83028F42B
:1006800001C09EE18FEF809362000093670090931A
:1006900061009AE086B3867011F49150D9F79923DE
:1006A00021F49093830090937D0091B39E50993FE5
:1006B0001CF481B78F5F81BF98301CF081B78150E7
:1006C00081BF8091600084FF1CC01123D1F0809114
:1006D000600084FF07C08091720098E889278093AA
:1006E000720003C08AE58093600080916600809369
:1006F000730061E083E790E045DD85E08093600072
:1007000003C0112309F0CFCE86B380958971109173
:0A0710006600182780936600C6CE2D
:04071A005A5AFF0028
:00000001FF
